:0200000480007A
:100000009710000093800000171100001301810178
:1000100083A1000013D2114093D2F14013D3F141D8
:1000200093D3014013D40141232031002322410006
:10003000232451002326610023287100232A8100F4
:1000400097100000938040FC17110000130101FF7E
:1000500003A40000935414401355F4409355F44105
:10006000135604409356044123208100232291001B
:100070002324A1002326B1002328C100232AD10074
:1000800097100000938080F817110000130181FC85
:1000900083A6000013D7164093D7F64013D8F64135
:1000A00093D8064013D906412320D1002322E10032
:1000B0002324F1002326010123281101232A2101F1
:1000C000171600001306C6F497160000938606FA6A
:1000D0000329060093591940135AF940935AF941DC
:1000E000135B0940935B094123A0260123A236013B
:1000F00023A4460123A6560123A8660123AA76015C
:1001000017160000130606F197160000938686F76F
:10011000832B060013DC1B4093DCFB4013DDFB410B
:1001200093DD0B4013DE0B4123A0760123A2860151
:1001300023A4960123A6A60123A8B60123AAC601DB
:10014000171D0000130D4DED971D0000938D0DF54B
:10015000032E0D00935E1E4013DF1E40935F1F4071
:1001600093D01F4013D110409351114023A0CD01D3
:1001700023A2DD0123A4ED0123A6FD0123A81D0078
:1001800023AA2D0023AC3D0097100000938000E9C6
:1001900017110000130141F283A2000013D0124096
:1001A0002320010097100000938080E717110000C2
:1001B0001301C1F083A2000013D0124093521040EB
:1001C000232001002322510017150000130585E5A7
:1001D00097150000938505EF370610F01306C6F259
:1001E0006306B5028326C5002320D600832685003A
:1001F0002320D600832645002320D6008326050031
:100200002320D600130505016FF09FFD370510F080
:10021000130505F223200500000000000000000087
:0402200000000000DA
:101000000000000001000000FFFFFFFFFFFFFF7F67
:101010000000008010EFCDAB7856341298BADCFE99
:10102000FFFFFFFFFFFFFFFFFFFFFFFFFFFFFFFFD0
:10103000FFFFFFFFFFFFFFFFFFFFFFFFFFFFFFFFC0
:10104000FFFFFFFFFFFFFFFFFFFFFFFFFFFFFFFFB0
:10105000FFFFFFFFFFFFFFFFFFFFFFFFFFFFFFFFA0
:10106000FFFFFFFFFFFFFFFFFFFFFFFFFFFFFFFF90
:10107000FFFFFFFFFFFFFFFFFFFFFFFFFFFFFFFF80
:10108000FFFFFFFFFFFFFFFFFFFFFFFFFFFFFFFF70
:10109000FFFFFFFFFFFFFFFFFFFFFFFFFFFFFFFF60
:1010A000FFFFFFFFFFFFFFFFFFFFFFFFFFFFFFFF50
:1010B000FFFFFFFFFFFFFFFFFFFFFFFFFFFFFFFF40
:040000058000000077
:00000001FF
